:04000000D9EF15F02F
:080008005FEF00F000000000B2
:100010000000000000000000046ED8CF05F0E0CF23
:1000200006F00001E9CF0CF0EACF07F0E1CF08F0CD
:10003000E2CF09F0D9CF0AF0DACF0BF0F3CF12F00C
:10004000F4CF13F0FACF14F0F5CF15F0F6CF16F089
:10005000F7CF17F000C00EF001C00FF002C010F093
:1000600003C011F09DA038EF00F09EB0DDEF01F06D
:100070000EC000F00FC001F010C002F011C003F07C
:100080000CC0E9FF07C0EAFF078E08C0E1FF09C006
:10009000E2FF0AC0D9FF0BC0DAFF12C0F3FF13C0A2
:1000A000F4FF14C0FAFF15C0F5FF16C0F6FF17C025
:1000B000F7FF045006C0E0FF05C0D8FF1000196E1E
:1000C000D8CF1AF0E0CF1BF00001E9CF21F0EACF42
:1000D0001CF0E1CF1DF0E2CF1EF0D9CF1FF0DACF38
:1000E00020F0F3CF27F0F4CF28F0FACF29F0F5CFA6
:1000F0002AF0F6CF2BF0F7CF2CF000C023F001C090
:1001000024F002C025F003C026F0F2A88BEF00F027
:10011000F2B2F2EF01F0F0A691EF00F0F0B0FBEFD9
:1001200001F0F0A897EF00F0F0B204EF02F0F2A6B1
:100130009DEF00F0F2B00DEF02F09DAAA3EF00F0EA
:100140009EBA45EF03F0A0AAA9EF00F0A1BA72EFA2
:1001500003F023C000F024C001F025C002F026C047
:1001600003F021C0E9FF1CC0EAFF1C8E1DC0E1FFA7
:100170001EC0E2FF1FC0D9FF20C0DAFF27C0F3FF77
:1001800028C0F4FF29C0FAFF2AC0F5FF2BC0F6FFF4
:100190002CC0F7FF19501BC0E0FF1AC0D8FF100099
:1001A0000101CB931F0ECC6FC86BC76BC853D8A48B
:1001B000A2D0C7510508D8A09ED0CA6B010EC96F46
:1001C000C751006E05E0D890C937CA37002EFBD75B
:1001D000C751006EC851036E035004E10052000184
:1001E00025E00101035005E1010E005C000123E060
:1001F0000101035005E1020E005C000121E0010154
:10020000035005E1030E005C00011FE001010350F3
:1002100005E1040E005C00011DE00101035005E151
:10022000050E005C00011BE0010121D00101CB9112
:1002300081A0CB811DD00101CB9181A2CB8118D0AF
:100240000101CB9181A4CB8113D00101CB9181A875
:10025000CB810ED00101CB9181AACB8109D00101C4
:10026000CB9180B4CB81CBA101D0898A01D000D0C1
:10027000640EC725016E010EC821036E640EC725EA
:10028000E96E010EC821EA6ED890EF34D06F000EEF
:10029000CBB1010ED01103C0EAFF01C0E9FFEF6E40
:1002A000640EC725E96E010EC821EA6EEF50CC1529
:1002B000C56F640EC725E96E010EC821EA6EEF50C6
:1002C000C515C66FCC51C65D06E1C9516213CA514E
:1002D0006313CB830CD0C65309E1CAC103F0031EDC
:1002E000C951FF0A62170350631701D0CB83C72B94
:1002F000D8B4C82B5BD76191CBB3618182B002D0F7
:10030000628D02D0629D636B80AC02D0628F02D09E
:10031000629F636B0001EDEF01F0D051FC0F3AE2F8
:10032000040FCCEF01F036D0D55302E1D65304E0F0
:10033000D551D8B4D607D507D5532BE1D65329E1EB
:10034000D05103080FE1D73D03D0D83D01D00AD0EA
:10035000D751D8B4D807D707D75304E1D85302E10F
:10036000D06B8A96D05103080AE1020ED06FD2C03A
:10037000D6F0D1C0D5F0CFA101D08A860AD0D05115
:10038000020807E1030ED06FD4C0D6F0D3C0D5F079
:100390008A9600D0EEEF01F0E824F76AF736B30F43
:1003A000F66E030EF7220A00F550FA6E0800F550BB
:1003B000F96E2603260328032803EC0ECF6E780E71
:1003C000CE6E898A010E0101606F0A0E5A27000E57
:1003D0005B235C235D230001E3D69FD7899A9E901F
:1003E00038EF00F00101605302E1040E606FF292F9
:1003F0000001A9EF00F00101605302E1040E606FFB
:10040000F0900001A9EF00F00101605302E1040E39
:10041000606FF0920001A9EF00F081CFD1F10101EE
:10042000605302E1040E606FF2900001A9EF00F04A
:10043000050E0101476FD4C1E9FFD5C1EAFFEFCF37
:1004400043F1ACBA01D0AC8AD4C1E9FFD5C1EAFF0F
:10045000EFCFADFF010ED425416F000ED521426FC5
:100460004007FC0E46150109466F405304E1FC0E9F
:1004700046150209466F00015FEF02F0060E01010A
:10048000476FACBA01D0AC8A010E036ED40EE96E90
:1004900003C0EAFFEFCFADFFD4C143F1FC0E461518
:1004A000466F000169EF02F001014651030B01089C
:1004B00008E142C1D5F141C1D4F10001B9D709D059
:1004C00001014651030B020805E145C1D4F10001C9
:1004D000D5D701010001B0EF02F001012B89D36BE8
:1004E000B8B2D32BD26BABCFD1F1060ED117D26BF2
:1004F000AECF4CF1D35301E04C6BD151D21139E165
:10050000D35337E1475105082EE143514C5D26E0B6
:10051000476BFC0E4615466F0D51010815E30D5152
:10052000030DF350D56BD46F010ED427000ED523E5
:10053000150ED425E96E010ED521EA6EEFCF00F03D
:1005400000380F0B010B03E10591058119832C5332
:1005500001E02B852DC12CF12B818ED00001A4D779
:1005600001018AD005D0475302E12B8901D03581A2
:1005700083D0D151020B006E036A0050031025E0B6
:10058000AB98476B0D51010815E30D51030DF35066
:10059000D56BD46F010ED427000ED523150ED425AC
:1005A000E96E010ED521EA6EEFCF00F000380F0B97
:1005B000010B03E10591058119832C5301E02B8583
:1005C0002DC12CF12B81AB8857D0D35307E1D151EA
:1005D000040B006E036A005003104EE04C5327E1F9
:1005E0004AA51CD00D51010815E30D51030DF35020
:1005F000D56BD46F010ED427000ED523150ED4254C
:10060000E96E010ED521EA6EEFCF00F000380F0B36
:10061000010B03E10591058119834A954AA704D08E
:100620000591058119834A97010E476F25D04751DF
:10063000020821E20D51010815E30D51030DF3509D
:10064000D56BD46F010ED427000ED523150ED425FB
:10065000E96E010ED521EA6EEFCF00F000380F0BE6
:10066000010B03E10591058119832C5301E02B85D2
:100670002DC12CF12B81476B000142EF03F09EAAA4
:1006800002D02BD79E9A4DEF03F08B860101605369
:1006900002E1020E606F0001F2D79E9AA9EF00F00E
:1006A0000101D56BD2C1D4F1D90ED225016E000E55
:1006B000D521036E01C0D6F1D76FD35302E0010EEE
:1006C00001D0000EE8B006D0D7C1EAFFD6C1E9FFDD
:1006D000EF9205D0D7C1EAFFD6C1E9FFEF82000152
:1006E00085EF03F00101605302E1060E606FD16BEC
:1006F00078BCD12BD15304E089988A968B968B9A3B
:10070000D26BD1C1D3F10001CBD7A19AA9EF00F0F0
:1007100001019D6B9D5314E19D51080DF3509F6B9A
:100720009E6F010E9E25016E000E9F21036E0150EB
:100730002E0FE96E000E0320EA6EEF909D2BEAD794
:1007400036C037F000011200C150F00BC16E010E2F
:100750000F01386F000E3C6F396F3A6F3B6FC0501E
:10076000C00B0709C06EC08EC28000011200D0DF2E
:100770002E6A316A050E306EE7DF43EF17F0010194
:100780009D51000A000101E004D0789E0F01416BE9
:1007900002D00F0100D001019F6BD90E9D25E96E9B
:1007A000000E9F21EA6EEF909F6BD90E9D25E96E9A
:1007B000000E9F21EA6EEF920001120001016C6BA6
:1007C0006C5307E16CC19DF10001D9DF01016C2B75
:1007D000F7D7000145EF17F0000EBA6EFF0EBB6EA3
:1007E000F00E0F015D178B9A0001120001016C6B76
:1007F0006C51010870E36C510A0DF3506E6B6D6F14
:10080000DA0E6D25E96E000E6E21EA6EEF6A6C510C
:100810000A0DF3506E6B6D6F010E6D25016E000EAB
:100820006E21036E0150DA0FE96E000E0320EA6EAE
:10083000EF906C510A0DF3506E6B6D6F020E6D25CB
:10084000016E000E6E21036E0150DA0FE96E000E8C
:100850000320EA6EEC6AED52EF6A6C510A0DF35018
:100860006E6B6D6F040E6D25016E000E6E21036EB2
:100870000150DA0FE96E000E0320EA6EEC6AED52C9
:10088000EF6A6C510A0DF3506E6B6D6F060E6D259D
:10089000016E000E6E21036E0150DA0FE96E000E3C
:1008A0000320EA6EEC6AED52EF6A6C510A0DF350C8
:1008B0006E6B6D6F080E6D25016E000E6E21036E5E
:1008C0000150DA0FE96E000E0320EA6EEC6AED5279
:1008D000EF6A6C2B8DD7899A899E0001EE6BEF6BC6
:1008E000F06BF26BF16BF46BF36BF66BF56BF86B13
:1008F000F76BFA6BF96B0F015E6B00016DDF47EF71
:1009000017F09D90D06B8A969D8092EF04F0CF8176
:10091000D06BD26BD16BD46BD36BD66BD56BD86BE2
:10092000D76BEFD749EF17F08B848B921200FCDF67
:100930004CEF17F089988B9857EF17F00400F2CF1F
:100940009CF1F29CF29E9BC1A9FFA69CA69EA6804C
:10095000A85001019CBDF28C9CBFF28E016E00017B
:1009600012000101836B050E846F836B8451835DDC
:100970002BE2040081C1A9FF82C1A8FFA69CA69E0C
:10098000A684F250006EF29CF29E0F01550EA76EE7
:10099000AA0EA76EA682A6B2FED7A6940050F212A7
:1009A000F2CF85F1F29CF29E81C1A9FFA69CA69E82
:1009B000A680A850010185BDF28C85BFF28E825DB4
:1009C00001E102D0832BD2D78451835D02E3000E74
:1009D00001D0010E016E0001120001017181020EB1
:1009E000726F72516E2771A114D0725312E06E07AC
:1009F0006EC181F16FC182F10001B3DF010171911C
:100A000001B0718171A104D0720770C16FF1706B78
:100A1000EAD7000E71B1010E016E000167EF05F01B
:100A200001017A5100D07A510001A803F350600F00
:100A300001017E6F00D07F6B7B517F5D15E27DC130
:100A400003F07CC1E9FF7DC1EAFFEFCF80F17EC1F9
:100A500081F180C182F1000184DF01017C2BD8B4D7
:100A60007D2B7E2B7F2BE8D700014FEF05F0010196
:100A70007269736974697569766977697869796982
:100A80006EC171F171516F5D0DE371C17AF170C189
:100A90007BF1010E7D6F720E7C6F0001C1D70101E9
:100AA000712BF0D700015DEF05F001016E6B090EAF
:100AB0006F6FA8C070F10001DAD776EF05F0120E63
:100AC00001016E6F706B0F0E6F6F000186D7110EF4
:100AD0000101816F0A0E826F000143DF180E0101D0
:100AE000816F060E826F00013CDFDFD7E8EF05F073
:100AF00001019D519F03F3CF01F0F4CF00F0A0035B
:100B0000F35000269E519F03F3500020026E000117
:100B10001200016A026A006A036A0101A85102E137
:100B2000A75118E0100EA96FD890A537A637003648
:100B30000336A851035C02E1A751005C07E3A7510B
:100B4000005ED8A00306A851035ED88001360236A5
:100B5000A92FEAD70001120001019B6B0001EEDE14
:100B600001C06CF1010E01019B6F0001E7DE01C0C5
:100B70006DF101016C51440803E16D2D01D035D0B8
:100B8000020E816F190E826F0001EBDE030E010170
:100B9000816F080E826F0001E4DE040E0101816F97
:100BA00082690001DEDE100E0101816F826B00019F
:100BB000D8DE050E0101816F010E826F0001D1DECA
:100BC000060E0101816F050E826F0001CADE77D724
:100BD0000101816B440E826F0001C3DE010E010131
:100BE000816F826F0001BDDE0101100E9B6F00015D
:100BF000A5DE01C06AF1020E01019B6F00019EDEBD
:100C000001016F6B01C06EF16FC19EF101C09DF1DA
:100C1000A06B9F6900016CDF02C06FF101C06EF133
:100C200002C0A6F101C0A5F10101A86B640EA76F77
:100C300000016FDF01C058F1030E01019B6F00013D
:100C40007DDE01016F6B01C06EF16FC19EF101C0CD
:100C50009DF1A06B9F6900014BDF02C06FF101C0E5
:100C60006EF102C0A6F101C0A5F10101A86B640EEE
:100C7000A76F00014EDF01C059F1060E01019B6F05
:100C800000015CDE01019E6B01C09DF1A06B640E52
:100C90009F6F00012DDF02C05FF101C05EF162EFC6
:100CA00017F06CC1EFF06DC1F0F068EF17F06DC197
:100CB000F6F06CC1F5F06EEF17F0CF9101016DA168
:100CC00003D00001CF81010100017AEF17F0040089
:100CD000F2CF71F1F29CF29E6CC1A9FFA69CA69E78
:100CE000A680A850010171BDF28C71BFF28E706BAD
:100CF0006F6B6E6B6D6F6FC170F16EC16FF16DC117
:100D00006EF16D6B010E6C25716FF2CF72F1F29C7A
:100D1000F29E71C1A9FFA69CA69EA680A85072BD96
:100D2000F28C72BFF28E6D136FC170F16EC16FF1F4
:100D30006DC16EF16D6B020E6C25716FF2CF72F1A9
:100D4000F29CF29E71C1A9FFA69CA69EA680A85007
:100D500072BDF28C72BFF28E6D136FC170F16EC1F5
:100D60006FF16DC16EF16D6B030E6C25716FF2CF7B
:100D700072F1F29CF29E71C1A9FFA69CA69EA6806C
:100D8000A85072BDF28C72BFF28E6D136DC100F06F
:100D90006EC101F06FC102F070C103F0000163EF9A
:100DA00007F00101715109083EE3725173113BE0F4
:100DB000715100D072C1E9FF73C1EAFFA8C0EFFF13
:100DC00071510001A803F350600F0101746F00D04E
:100DD000756B72C1E9FF73C1EAFFEF50755D23E2E5
:100DE000010E7225E96E000E7321EA6EECCF77F1E9
:100DF000ED52EFCF76F1036A75517625016E77518A
:100E0000032201C078F103C079F174C19BF10001A4
:100E100095DD79C1EAFF78C1E9FF01C0EFFF01016B
:100E2000742B752BD6D7000151EF07F001016E6BC3
:100E3000580E6D6F6C6B6C51090836E36C51030DE5
:100E4000F350706B6F6F010E6F25016E000E7021F5
:100E5000036E01503A0FE96E000E0320EA6E6EC178
:100E6000ECFFED526DC1EFFF6C5100D00001A851B5
:100E700001016D27000E6E2300D06C51030DF3505D
:100E8000036A3A0F016E000E032201C06FF103C026
:100E900070F16CC171F103C073F101C072F1000116
:100EA00080D701016C2BC7D700016CEF07F0180E3B
:100EB00001019B6F000142DD01C0A8F0140E010189
:100EC0006C6F000104D703C0ACF002C0ABF001C0EE
:100ED000AAF000C0A9F0AAD77CEF17F001019D533A
:100EE0000AE0D56AF29A370ECD6ECC6A9D92B46A4A
:100EF000B16AA09204D0CD6ACC6A9D909E90000108
:100F00001200948C0F013A9D948E3A9FAB98AB9E41
:100F1000AC84B886B898B892B890AB88AC98AC9AC4
:100F2000AC96CF0EAF6EB06AAB8E9E9AAECF4CF140
:100F3000AECF4CF101014C6BD08E9F8AF28C9E9A01
:100F40009F8AF28E000112008B86A9EF07F0D9DF8D
:100F5000FBD70101476B0001B2EF07F001016C6B99
:100F60000001F5D70101346B336B010E0E6F146F66
:100F70009A0E0F6F106B116B010E126F136B6C6B6F
:100F80006C51070812E3036A6C511B0FE96E010EE6
:100F90000320EA6EEF68036A6C51230FE96E010EBD
:100FA0000320EA6EEF686C2BEBD72C6B2B6B2F6B4F
:100FB0000001DCEF07F0D2D7000E016EEFEF07F073
:100FC000CF930101B7A103D00001CF83010100013C
:100FD000CFA302D09D8A01D09D9A1200ECD70101C7
:100FE000B86B010EB76F0001EBDF85EF17F09D9036
:100FF0005DC1AFF15CC1AEF15BC1ADF15AC1ACF105
:101000009D80ACC100F0ADC101F0AEC102F0AFC136
:1010100003F012000400F2CF9EF1F29CF29E9BC1FD
:10102000A9FFA69CA69EA680A85001019EBDF28C99
:101030009EBFF28E9D6B9C6F9CC19DF19C6B010EBF
:101040009B259E6FF2CF9FF1F29CF29E9EC1A9FF5D
:10105000A69CA69EA680A8509FBDF28C9FBFF28E34
:101060009C139CC101F09DC102F000019AEF11F0A8
:1010700001016251B315006E6351B415036E00C0D7
:1010800001F0026E000112009D900101A051A1111A
:1010900003E1A251A31133E0040E0001EE6FA1C1E0
:1010A000A6F1A0C1A5F10101A86B0A0EA76F00016E
:1010B00030DD02C0F2F001C0F1F0A3C1A6F1A2C17F
:1010C000A5F10101A86B0A0EA76F000122DD02C085
:1010D000F4F001C0F3F0F2C0F8F0F1C0F7F0010154
:1010E000A45303E10368FF0E02D0036AA451000178
:1010F000F96F03C0FAF0EFC05EFF10D00101010EDE
:101100000001EE6FF26BF16BF46BF36BF6C0F8F06D
:10111000F5C0F7F0FA6BF96BF0C05EFF9D8012002E
:101120000101B26BB46B1F0EB36F0001A1DF02C0EF
:10113000B4F101C0B3F10101B151015C29E1B45333
:1011400027E1B151010A000109E0030A0CE0060A97
:101150000FE00C0A12E0180A15E019D0010E010187
:10116000B26F000114D0020E0101B26F00010FD066
:10117000030E0101B26F00010AD0040E0101B26F2B
:10118000000105D0050E0101B26F000100D0010180
:10119000B2C101F000015FEF09F0BBC1C1F1BAC1FA
:1011A000C0F1BDC1C3F1BCC1C2F10101BF5303E134
:1011B000BE51000830E2C0C1E9FFC1C1EAFFEFCF74
:1011C000C4F1C3C103F0C2C1E9FFC3C1EAFFEF50DC
:1011D000C45D16E0C1C103F0C0C1E9FFC1C1EAFFAF
:1011E000EFCFC4F1C3C103F0C2C1E9FFC3C1EAFF3D
:1011F000EF50C45D02E2FF0E01D0010E016E0DD072
:10120000C02BD8B4C12BC22BD8B4C32BBE51D8B479
:10121000BF07BE07CBD7000E016E0001E7EF09F054
:10122000200ED8800101B155036AAD0F016E000E8A
:10123000032201C0B3F103C0B4F1B66BAD0EB56FBC
:10124000B26BB151B25D1CE2B6C103F0B551B52B22
:10125000D8B4B62BB76F03C0B8F1B4C103F0B35123
:10126000B32BD8B4B42BE96E03C0EAFFEFCFB9F1CA
:10127000B8C1EAFFB7C1E9FFB9C1EFFFB22BE1D7AF
:10128000B1C1CDF0000101EF0AF00101AD69AE6B13
:10129000AB51FF080DE0ABBF08D0AB510001CD5DF5
:1012A000D8B002D0010104D00101FE0EAD6FADD067
:1012B000AC53D8B4AAD0ACC1B1F1000131D701C050
:1012C000AEF10101AE53D8B4A0D0036A0001CD51F4
:1012D000AD0FE96E000E0320EA6EAEC1EFFFCD2B1D
:1012E0000101AF6BAA51AF5DD8B079D0036AAF519D
:1012F000A825E96EA9510320EA6EEFCFB0F1B051F5
:10130000030DF350B26BB16F3A0EB125E96E000ECA
:10131000B221EA6EEF525FE0B051030DF350B46BAF
:10132000B36F3A0EB325E96E000EB421EA6EEF50AA
:101330000001CD5DD8B002D001014DD00101B05106
:10134000030DF350B26BB16F010EB125016E000EAB
:10135000B221036E01503A0FE96E000E0320EA6ECF
:10136000ECCFB2F1ED52EFCFB1F1B051030DF3502C
:10137000B46BB36F3A0EB325E96E000EB421EA6E7A
:10138000EF500001CD5D036AAD0F016E000E032228
:1013900001C0B5F1010103C0B6F1B051030DF35026
:1013A000B86BB76F3A0EB725E96E000EB821EA6E3A
:1013B000EFCFB9F1B2C1BBF1B1C1BAF103C0BDF118
:1013C00001C0BCF1BF6BB9C1BEF10001E6D601524C
:1013D00003E1010104D000010101AF2B83D7AA5121
:1013E000AF5D03E2AFC1ADF110D0AB510001CD5DF7
:1013F0000DE10101AB51FF0806E1070EB16F0001DD
:101400000FD704D00101FE0EAD6F00010101ADC187
:1014100001F0000130EF0AF001019C6B010E9D6F9D
:10142000020E9E6F030E9F6F040EA06F050EA16F3C
:10143000060EA26F070EA36F080EA46F090EA56F0C
:101440003A50040DF3CFA7F1010EA96F9C0EA86FBF
:101450000A0EAA6FA7C1ABF19BC1ACF1000115D771
:1014600001C0A6F10101A6BF0CD00001CD6B036A3B
:101470000101A6519C0FE96E010E0320EA6EEFCF29
:10148000A6F1A6C101F00001A8EF12F0ADC132F142
:1014900032C14EF1ACC14DF1030E0101476F4A83D9
:1014A000496B000112000101B7910001CFA303D0E5
:1014B0000101B78100019D9ACF93000E0101B7B1E0
:1014C000010E036A016E03C002F000011200050E56
:1014D0000101476FB7C1E9FFB8C1EAFFEFCF43F1A0
:1014E000ACBA01D0AC8AB7C1E9FFB8C1EAFFEFCF0F
:1014F000ADFF010EB725416F000EB821426F4007C6
:10150000FC0E46150109466F405304E1FC0E4615DA
:101510000209466F0001F2EF0AF00101B56BB46BEE
:10152000B66B446B050E476FB3C140F1B3C132F1E6
:10153000B051140804E1506B36C14FF102D0506B2A
:101540004F6B0001B0DF02C031F101C030F1010189
:10155000B56BB46BB5531BE1B351B45D18E2370EF4
:10156000B425016E010EB521036EB151B425E96EAB
:10157000B251B521EA6EEFCFB9F103C0EAFF01C065
:10158000E9FFB9C1EFFFB42BD8B4B52BE3D731C114
:10159000B8F130C1B7F1000113DD010E0101405D6A
:1015A0004B6F010E526F370E516F036A4B5151252D
:1015B000E96E52510320EA6EEF504F27000E502380
:1015C0005051B66FB6514F27000E5023506B4B53FE
:1015D00003E14FC145F1451F010EB86F370EB76FDC
:1015E000000175D701014A85000112000101AA6BB3
:1015F000A96BA7C12DF1A7513C0A000107E0410AE0
:1016000011E0830A21E0410A20E020D0FB0E010115
:101610000D6FA7C136F10D0EAC6F080EAD6F000156
:1016200035DF85D001012E530DE02E6BA7C136F1B9
:101630000D0EB06F010EB26F230EB16F080EB36FB7
:1016400000016BDF000173D072D071D0010E010177
:10165000AA6F150EA96FA86BA851010865E3AAC16E
:1016600003F0A9C1E9FFAAC1EAFFA751EF5C55E168
:10167000A8C10DF1010EA925016E000EAA21036E6D
:1016800001C0E9FFEA6EEFA032D02DC136F1A851BA
:10169000080DF350AC6BAB6FFD0EAB25016E000E69
:1016A000AC21036E01C0ADF1AE6F020EA925016E33
:1016B000000EAA21036E01C0E9FFEA6EEFCFAFF181
:1016C000140EB06FAEC1B2F1ADC1B1F1AFC1B3F1A3
:1016D000000123DF010E0101A925016E000EAA21E0
:1016E00001C0E9FFEA6EEF50FD0BEF6E14D02DC183
:1016F00036F1020EA925016E000EAA21036E01C06B
:10170000E9FFEA6EEFCFABF1140EAC6FABC1ADF1F8
:101710000001BCDE01010CD001D00D69030EA92728
:10172000000EAA23A82B98D7476B000100D0010117
:10173000000121EF0DF001012E6B0001E2EF0CF032
:1017400001010D51FF0A000103E0040A02E038D054
:1017500093D001012C5301E02B852DC12CF12B835B
:101760000001A1DE02C031F101C030F10101A76B1F
:101770003251A75D1BE2036AA7511B0F016E010ED8
:10178000032201C0A8F103C0A9F1036AA751370FD2
:10179000E96E010E0320EA6EEFCFAAF1A9C1EAFFBC
:1017A00001C0E9FFAAC1EFFFA72BE2D731C1B8F111
:1017B00030C1B7F1000104DC01012F8100015CD0D0
:1017C00001012C5301E02B852DC12CF12B8300014D
:1017D0006ADE02C031F101C030F10101A76B325164
:1017E000A75D25E20D51080DF350A96BA86F036AA0
:1017F000A751A825016EA95103220150FD0F016ECA
:10180000000E032201C0A8F103C0A9F1036AA75189
:10181000370FE96E010E0320EA6EEFCFAAF1A9C1DE
:10182000EAFF01C0E9FFAAC1EFFFA72BD8D731C15A
:10183000B8F130C1B7F10001E0EC07F001010D5142
:10184000030DF350A96BA86F010EA827000EA92362
:10185000150EA825E96E010EA921EA6EEF820D5141
:10186000000A000103E0010A03E004D0FB6903D091
:10187000FC6901D000D000D0EFEF0CF001012C5337
:1018800001E02B852DC12CF12B8318512D5D02E138
:10189000059119830D51010810E30D51030DF3500B
:1018A000A86BA76F010EA727000EA823150EA7256A
:1018B000E96E010EA821EA6EEF92000121EF0DF012
:1018C0000101A66B4751000A00010CE0010A0BE080
:1018D000030A23E0010A28E0070A5BE0020AD8B401
:1018E00080D0AED0AED001014C51550803E1020EBC
:1018F000476F11D0000181EC07F00101476B2C53B9
:1019000001E02B852DC12CF12B814AA704D0059134
:10191000058119834A97000194D00101476B4CC19E
:10192000A7F1000163D68DD001014E51325D036AEB
:10193000370FE96E010E0320EA6E4CC1EFFF4A83B8
:101940004A854A87496B4E51325D09E14D51140871
:1019500004E1506B36C14FF102D0506B4F6B4E51CA
:10196000325D036A370FE96E010E0320EA6EEF5015
:101970004F27000E50235051A66FA6514F27000E3F
:101980005023506B4E074E5302E1040E476F000187
:1019900058D04CC13FF1010150C103F0031E4F511B
:1019A000FF0A506B4F6F4A934A954A97496B476BB2
:1019B0004F514C5D02E1505310E02D513C0803E1C2
:1019C0000001B9D601010591058119832C5301E06D
:1019D0002B852DC12CF12B8102D00001B1D6000145
:1019E00030D001014A9543514C5D26E0476BFC0E17
:1019F0004615466F0D51010815E30D51030DF350C7
:101A0000A86BA76F010EA727000EA823150EA72508
:101A1000E96E010EA821EA6EEFCF00F000380F0B3F
:101A2000010B03E10591058119832C5301E02B85FE
:101A30002DC12CF12B8106D0476B00011FD701D09F
:101A400000D001010001120001014B07036A4B5154
:101A50005125E96E52510320EA6EEF504F27000ED8
:101A600050235051A66FA6514F27000E5023506BA4
:101A70004B5305E14FC145F1451F506B4F6B0001C2
:101A800012002CC1A7F12BC1A6F101012C6B2B6B0D
:101A9000A6C101F0A7C102F0000112000101A9C115
:101AA000E9FFAAC1EAFFA9C0EFFF0001DDEF0DF0D9
:101AB00001011D51B00A000112E0020A3EE0010AD4
:101AC000D8B49BD0070AD8B49AD0010AD8B4B3D0FE
:101AD000030AD8B4B2D0010AD8B4CAD03CD10101AB
:101AE00014511B5D29E11C51060826E10F511E5DB2
:101AF00003E01E517F0820E110511F5D02E01F3DF1
:101B00001BD01151205D02E0203D16D01251215D05
:101B100002E0213D11D022C10EF114C123F1010ECA
:101B2000246F400E1D25256F2669276928692969BC
:101B30002A69010E2E6F00D011D1010114511B5DD5
:101B400003E114510E5D58E11C51060855E10F5197
:101B50001F5D02E01F3D50D01051205D03E0205179
:101B60007F084AE11151215D02E0213D45D012512B
:101B7000225D02E0223D40D01E51000A000103E038
:101B8000010A14E025D00EC123F1060E0101246FD5
:101B9000400E1D25256F0FC126F110C127F111C17F
:101BA00028F112C129F113C12AF121D0010E01013E
:101BB000AA6F260EA96F000171D70EC123F1050E81
:101BC0000101246F400E1D25256F2A6910D00001E8
:101BD0000EC123F1030E0101246F7F0E256F1DC17D
:101BE00026F1120E276F286929692A6900D0010E93
:101BF0002E6F346B336B00D0B1D00101AFD0010137
:101C000014511B5D03E114510E5D14E11C510608D3
:101C100011E10EC123F1030E246F7F0E256F1DC14C
:101C200026F1120E276F286929692A69010E2E6F85
:101C3000346B336B93D0010191D0010114511B5DC2
:101C400003E114510E5D13E11C2D11D00EC123F1DF
:101C5000030E246F7F0E256F1DC126F1120E276F14
:101C6000286929692A69010E2E6F346B336B76D08F
:101C7000010114511B5D03E114510E5D6BE11C5118
:101C8000060868E1A66BA76B040EA66FA65310E0CA
:101C9000036AA6511E0FE96E010E0320EA6EEF3CA7
:101CA00001D004D0010EA65DA76F02D0A607EED723
:101CB000A7511E2501080EE20EC123F1030E246F69
:101CC0007F0E256F1DC126F1120E276F2869296925
:101CD0002A693CD01EC1A8F1A66BA651A75D2AE3D4
:101CE000010EA625036A1E0FE96E010E0320EA6E9F
:101CF000EF3C01D01DD0A651A825030DF350AA6BCF
:101D0000A96F150EA925016E010EAA21036EAC6FF5
:101D1000010EA625036A1E0FE96E010E0320EA6E6E
:101D2000EFCFADF1ACC1EAFF01C0E9FFADC1EFFFFC
:101D3000A62BD3D70EC123F1010E246F400E1D2513
:101D4000256F26692769286929692A69010E2E6F7E
:101D5000346B336B03D001012E6B00D000015DEFBB
:101D60000FF001011D51B00A00010DE0020A27E049
:101D7000010A27E0070A27E0010A27E0030A27E013
:101D8000010A27E06BD001011C51060817E10F5131
:101D90001E5D03E01E517F0811E110511F5D02E03E
:101DA0001F3D0CD01151205D02E0203D07D01251A3
:101DB000215D02E0213D02D022C10EF151D001018E
:101DC0004FD001014DD001014BD0010149D001019B
:101DD00047D001011C51060840E1A66BA76B040E19
:101DE000A66FA65310E0036AA6511E0FE96E010EFE
:101DF0000320EA6EEF3C01D004D0010EA65DA76F70
:101E000002D0A607EED7A7511E25010801E225D072
:101E10001EC1A8F1A66BA651A75D1FE3A651A82578
:101E2000030DF350AA6BA96F150EA925016E010EC3
:101E3000AA21036EAC6F010EA625036A1E0FE96E80
:101E4000010E0320EA6EEFCFADF1ACC1EAFF01C095
:101E5000E9FFADC1EFFFA62BDED702D0010100D014
:101E6000000181EF0FF001012E530AE0332BD8B4AB
:101E7000342B345303E13351320801E22E6B02D08C
:101E8000346B336B2FA140D02F911B517E0801E0A2
:101E90002E6B0E511B5D06E01B517F0803E01451B1
:101EA0001B5D1DE11C51F00B17E11D51AF0807E24E
:101EB0001D51B70804E30001FBD50FD001010EC18D
:101EC00023F1030E246F7F0E256F1DC126F1100E26
:101ED000276F286929692A69000117D001011B535E
:101EE00002E12B8711D01B517E080DE11C51F00B34
:101EF00009E11D51AF0806E21D51B70803E30001D7
:101F000030D7010101D02E6B00011200010EEA6EE4
:101F1000A80EE96EEF5011E0050E016EBF0E006EC7
:101F20000400002EFDD7012EF9D72E0E006E002ED4
:101F3000FED700000400EF2EEFD71FEF14F08B84C4
:101F40008B8246EF14F08B948B926AEF14F08B9493
:101F50008B826DEF14F0D8B204D0010EEA6EAF0E92
:101F6000E96E006A016A026A036A0101AF6BB06B35
:101F7000B16BB26BAE51AD11AC11AB112CE0200EB8
:101F8000B36FD890A737A837A937AA37AF37B0377C
:101F9000B137B237AE51B25D08E1AD51B15D05E187
:101FA000AC51B05D02E1AB51AF5D0FE3AB51AF5F40
:101FB000AC51D8A0AC3DB05FAD51D8A0AD3DB15F44
:101FC000AE51D8A0AE3DB25FD880003601360236A1
:101FD0000336B32FD6D7AFC1EFFFB0C1ECFFB1C10D
:101FE000ECFFB2C1ECFF0001FFEF14F00101AF6B99
:101FF000B06B010EB16FDA6AD96AB46FA70EB36F16
:10200000010EEA6EAB0EE96EB4C1E2FFB3C1E1FFAF
:10201000B1C1B2F1D890E550EE02F350AF23F450C5
:10202000B023B22FF7D7AFC1DEFFB0C1AFF1B06BB5
:10203000D8B0B02BB32BD8B4B42BB12BB151050809
:10204000DFE1000119EF15F09D90EE5304E1010E60
:10205000EE6FF0C05EFFEE2D04D0F6C0F8F0F5C0D4
:10206000F7F09D8028EF11F001019E510A0DF35009
:10207000A06B9F6FDA0E9F25E96E000EA021EA6E1D
:10208000EF50020825E09E510A0DF350A26BA16F9C
:10209000DA0EA125E96E000EA221EA6EEF500308C8
:1020A00017E09E510A0DF350A46BA36F060EA325F3
:1020B000016E000EA421036E0150DA0FE96E000ECE
:1020C0000320EA6EEF5204E1EC5202E1000E01D06F
:1020D000010E016E00011200D05302E1000E01D08A
:1020E000010E016E9BEF10F0EE5302E0000E01D0E6
:1020F000010E016EA1EF10F001019D51020803E1F4
:10210000020E576F27D09D2D01D01ED061B11CD07B
:102110009E6B0001A9DF0152D8B402D0010114D096
:10212000010E01019E6F00019FDF0152D8B402D061
:1021300001010AD0D1D70152D8B402D0010104D094
:10214000D3D7015205E10101010E576F03D0000101
:102150000101576B00012BEF11F0C29088EC03F0E6
:1021600033EF11F0B8828B9652EF11F001019F6BA3
:102170009DC19EF1D90E9D25E96E000E9F21EA6E4C
:10218000EFB040D09D51000A000101E031D0800E37
:102190000F01416F1F0E406F040E776E940E786E24
:1021A000796A92500109926E9350040000D00000A9
:1021B00001019F6B9DC19EF1D90E9D25016E000E00
:1021C0009F21036E01C0A0F1A16F78AC02D0010E77
:1021D00001D0000EE8B006D0A1C1EAFFA0C1E9FF1E
:1021E000EF9205D0A1C1EAFFA0C1E9FFEF8202D0C2
:1021F000010100D09F6BD90E9D25E96E000E9F2135
:10220000EA6EEF80000162EF11F0000E0509BA6E70
:10221000FF0EBB6E8A9A0C0E0F015D6F5C6B5B6BE1
:10222000010E5A6F3F0E4917000E491300017CEF53
:1022300011F08B867DEF11F004000101B46B7F0E6D
:10224000B36F000138EC08F00150021001E0FCD639
:102250009BC19DF151D701015751020853E0606BBA
:10226000D19000017AD7010157531DE181CF9CF134
:10227000F290F292F0909D6B00016EEC07F0ECECA6
:1022800003F08998A19AA09A01019D6B0001BFEC0F
:1022900003F04F0E926EF70E936E810E946EF288DD
:1022A000F08660D70101605309E1575302E1000E47
:1022B00001D0010ED39EE8B0D38E030000009D6BC9
:1022C000000154D7A08A0101575317E1626AF298BE
:1022D000F0964F0E926EF70E936E370E616EF19E72
:1022E000810E946E6181010E9D6F00016EEC07F00E
:1022F000CF68CE689D8089D79CD70001A4EC03F0FD
:10230000D180010100013DEF15F001016C6B6D6B97
:102310006F6B0001F7EC07F003C08BF102C08AF18C
:1023200001C089F100C088F1120E01019B6F00010C
:102330000AEF08F002C09CF1010101C09BF1030EFD
:102340009E6FE80E9D6F02C0A0F101C09FF10001D9
:1023500078EC05F001018F6B8E6B02C08DF101C02E
:102360008CF1110E9B6F00019EEC04F00101976B44
:10237000966B956B01C094F16C510308D8B4D6EFFD
:1023800015F098810001F7EC07F003C07BF102C063
:102390007AF101C079F100C078F101016C51000AB5
:1023A000000106E0010A32E0030AD8B442D163D149
:1023B000CD6B0101B46B1F0EB36F000138EC08F058
:1023C00001C06EF17BC173F17AC172F179C171F113
:1023D00078C170F17BC187F17AC186F179C185F14D
:1023E00078C184F197C193F196C192F195C191F1B1
:1023F00094C190F1010E01016C6F7BC17FF17AC134
:102400007EF179C17DF178C17CF137D11F0E0101D8
:102410009B6F010E9C6F9D6B6EC19EF1B46B9BC157
:10242000B3F1000138EC08F001C06EF101019E51DA
:102430006E5D12E06E519E199D6F6E519D179D53FA
:102440000BE0A16B320EA06FA36BA26B010EA46F09
:10245000000144EC08F001019DC101F001C06FF1E1
:102460006F5308E097C193F196C192F195C191F134
:1024700094C190F19C6B6EC19BF19E6B180E9D6F89
:10248000A26BA16B010EA06FF40E9F6FA36B9B5309
:1024900002E19C5306E09D519B5D03E19E519C5DD2
:1024A0000DE00001F7EC07F003C087F102C086F1F0
:1024B00001C085F100C084F12DD001010001F7ECCD
:1024C00007F003C0A7F102C0A6F101C0A5F100C04A
:1024D000A4F101018451A45DA86F8551A559A96F8C
:1024E0008651A659AA6F8751A759AB6FA251AB5D10
:1024F0000FE30BE1A151AA5D0BE307E1A051A95D38
:1025000007E303E1A8519F5D03E2020EA36F02D02F
:10251000010EA36F0101A3C101F00150020813E1F4
:102520000001CD6B030E01016D6F010EA16FF40E62
:10253000A06FA36BFA0EA26F030EA46F000144EC10
:1025400008F03ED001016FC19BF100010CEF0AF0D1
:1025500001C09AF101019A51FE081AE10001CD6B08
:10256000020E01016C6F7BC17FF17AC17EF179C1EE
:102570007DF178C17CF1A16BFA0EA06FA36B780E90
:10258000A26F050EA46F000144EC08F019D0010100
:102590009ABF17D09ABF03D09A51090812E30001DD
:1025A000CD6B020E01016D6F010EA16FF40EA06FD5
:1025B000A36BFA0EA26F030EA46F000144EC08F0A7
:1025C00001010001CD5333E077C19EF176C19DF149
:1025D00075C19CF174C19BF101019F919E51935D66
:1025E00015E30BE19D51925D11E307E19C51915D73
:1025F0000DE303E190519B5D09E29B51905F9C517B
:10260000915B9D51925B9E51935B05D0936B926B56
:10261000916B906B9F81000E9FB1010E016E015274
:1026200004E00001CD6B03D001019891000101018C
:1026300024D001017C51785D9B6F7D5179599C6F4D
:102640007E517A599D6F7F517B599E6F8F519E5D50
:102650000EE30BE18E519D5D0AE307E18D519C5D18
:1026600006E303E18C519B5D02E36C6B03D0989110
:102670006F6B6E6B02D0010100D07851D00809E178
:102680007951070806E17A5304E17B5302E1030E16
:102690006D6F7851A00809E179510F0806E17A536E
:1026A00004E17B5302E1020E6D6F010E9B6F00018E
:1026B000F7EC07F003C0A1F102C0A0F101C09FF147
:1026C00000C09EF1010135A105D0000160EC0CF0C5
:1026D000010135914B5304E0000124EC0DF00101A0
:1026E000000141EC0DF002C09DF101C09CF101011F
:1026F0009CC100F0036A9C5103100AE0A1C18BF158
:10270000A0C18AF19FC189F19EC188F1020E9B6F21
:10271000000133EC0FF001014AA32FD0492B49519E
:1027200000082BE2476B000181EC07F001014AA78A
:1027300004D00591058119834A974AA51CD04A9572
:102740000D51010815E30D51030DF350A36BA26F5A
:10275000010EA227000EA323150EA225E96E010E7D
:10276000A321EA6EEFCF00F000380F0B010B03E15D
:102770000591058119834A93496B4AA10BD0482BD7
:102780004851000807E2476B000181EC07F00101A6
:102790004A91486B9CB71BD088519E5DA26F8951AE
:1027A0009F59A36F8A51A059A46F8B51A159A56F4E
:1027B0005651A55D0CE30BE15551A45D08E307E11B
:1027C0005451A35D04E303E15351A25D00E39BC1B7
:1027D00001F001C099F16D51020803E06D51030849
:1027E00004E1995301E18B8803D0995301E08B9860
:1027F0000001F7EC07F003C09EF102C09DF101C09B
:102800009CF100C09BF101016D51020803E06D5184
:10281000030816E1000194EC04F0898801016D5170
:10282000020802E1010E01D0020E0001CE6F040E7B
:1028300001016D6F010EA86F000186EF0FF001011D
:102840006D51000A00010FE0010A0DE0060A0BE0DD
:10285000050A0AE0010A08E0070A07E0010A1BE08E
:10286000030A3DE088D088D087D00101B46B400EC8
:10287000B36F000138EC08F00150021005E0070EBC
:1028800001016D6F06D000019FEF0FF0050E0101F1
:102890006D6F000171D00101B46B400EB36F000188
:1028A00038EC08F00150021005E0070E01016D6FD1
:1028B00014D00001060E01016D6F9EC183F19DC110
:1028C00082F19CC181F19BC180F10001CE2D03D02A
:1028D000A3EF0FF002D0A7EF0FF000014DD00101E0
:1028E000B46B400EB36F000138EC08F001500210D9
:1028F00005E0070E01016D6F3CD00001CE2D07D021
:10290000EE0E006E020E016E026A036A06D0EE0E33
:10291000006E020E016E026A036A03C0A2F102C0D9
:10292000A1F101C0A0F100C09FF1010180519B5DA8
:10293000A36F81519C59A46F82519D59A56F8351FA
:102940009E59A66FA251A65D14E30BE1A151A55DAE
:1029500010E307E1A051A45D0CE303E19F51A35DE7
:1029600008E30001CE2D02D0010E01D0000E0101BE
:102970006D6F000101D000D001016D51070A000107
:1029800005E0070A04E0010A02E005D0898E94EC14
:1029900004F0899801D000D00101A26BA16BA06B5B
:1029A0009F6B0001F7EC07F001017051005C9B6F19
:1029B000715101589C6F725102589D6F73510358A9
:1029C0009E6F9E530AE19D5308E19C5102083AE232
:1029D000FF0A03E19B51E70835E2D8929EC1AAF1B4
:1029E0009DC1A9F19CC1A8F19BC1A7F1AE6BAD6BD4
:1029F000030EAC6FE80EAB6F0001ABEF0FF003C03E
:102A0000A2F102C0A1F101C0A0F100C09FF1A2C1DA
:102A1000AAF1A1C1A9F1A0C1A8F19FC1A7F101012B
:102A2000AE6BAD6B030EAC6FE80EAB6F0001F6EF53
:102A30000FF00050010170270150712302507223E2
:102A4000035073239FC100F0A0C101F0A1C102F0A7
:102A5000A2C103F003C077F102C076F101C075F1A5
:102A600000C074F1995304E198B102D0010E996F3E
:102A700099C19BF100011CEF11F0010E01019B6F48
:102A80000001F7EC07F003C0A1F102C0A0F101C002
:102A90009FF100C09EF1010135A105D0000160EC5D
:102AA0000CF0010135914B5304E0000124EC0DF0D2
:102AB0000101000141EC0DF002C09DF101C09CF14B
:102AC00001019CC100F0036A9C5103100AE0A1C1FE
:102AD0008BF1A0C18AF19FC189F19EC188F1020EDC
:102AE0009B6F000133EC0FF001014AA32FD0492B5B
:102AF000495100082BE2476B000181EC07F001010E
:102B00004AA704D00591058119834A974AA51CD08C
:102B10004A950D51010815E30D51030DF350A36BB8
:102B2000A26F010EA227000EA323150EA225E96EA7
:102B3000010EA321EA6EEFCF00F000380F0B010B5E
:102B400003E10591058119834A93496B4AA10BD092
:102B5000482B4851000807E2476B000181EC07F061
:102B600001014A91486B9CB71BD088519E5DA26FB2
:102B700089519F59A36F8A51A059A46F8B51A159B4
:102B8000A56F5651A55D0CE30BE15551A45D08E31B
:102B900007E15451A35D04E303E15351A25D00E357
:102BA0009BC101F001C099F1BCEF11F0000187EF6A
:102BB00017F0F86A9F90F08CF08EF1809F8AA28ABD
:102BC000D08E078EEA6AE96A700ED36E9B9C9B9E3C
:102BD000366836C037F0CD6BCE6B01014C6B476B5E
:102BE0004D6B4E6B486B496B506B4F6B4B6B526B25
:102BF000516B0D692D6B316B306B2E6B326B566BDD
:102C0000556B0F0E546FA00E536F0001CF9301014F
:102C10005D6B5C6B5B6B5A6B6B6BC150F00BC16E89
:102C2000000E0F01386F3C6F396F3A6F3B6F776A58
:102C3000786A796A2E6A2F6A306A316A326A336A30
:102C4000346A356A386A396A3A6A3B6A3C6A3D6A6C
:102C50003E6A3F6A406A416A426A436A446A456A18
:102C6000466A476A486A496A4A6A4B6A4C6A4D6AC8
:102C70004E6A4F6A506A516A526A536A546A556A78
:102C8000566A576A586A596A5A6A5B6A5C6A5D6A28
:102C90005E6A5F6A0001606B616B626B636B646BA1
:102CA000656B666B676B686B696B6A6B6B6B6C6B88
:102CB0006D6B6E6B6F6B706B716B726B736B746B38
:102CC000756B766B776B786B796B7A6B7B6B7C6BE8
:102CD0007D6B7E6B7F6B806B816B826B836B846B98
:102CE000856B866B876B886B896B8A6B8B6B8C6B48
:102CF0008D6B8E6B8F6B906B916B926B936B946BF8
:102D0000956B966B976B986B996B9A6B9B6B9C6BA7
:102D10009D6B9E6B9F6BA06BA16BA26BA36BA46B57
:102D2000A56BA66BA76BA86BA96BAA6BAB6BAC6B07
:102D3000AD6BAE6BAF6BB06BB16BB26BB36BB46BB7
:102D4000B56BB66BB76BB86BB96BBA6BBB6BBC6B67
:102D5000BD6BBE6BBF6BC06BC16BC26BC36BC46B17
:102D6000C56BC66BC76BC86BC96BCA6BCB6BCC6BC7
:102D7000CF91D06BD16BD26BD36BD46BD56BD66B41
:102D8000D76BD86BD96BDA6BDB6BDC6BDD6BDE6B17
:102D9000DF6BE06BE16BE26BE36BE46BE56BE66BC7
:102DA000E76BE86BE96BEA6BEB6BEC6BED6BEE6B77
:102DB000EF6BF06BF16BF26BF36BF46BF56BF66B27
:102DC000F76BF86BF96BFA6BFE0EFD6FFE6FFF6928
:102DD000010100690169026903690469056F066FF1
:102DE0000769086909690A690B690C69356B366BF3
:102DF000376B386B396B3A6B3B6B3C6B3D6B3E6BA7
:102E00003F6B406B416B426B436B446B456B466B56
:102E10004A6BC10E156F810E166F020E176F420EB0
:102E2000186F810E196F080E1A6F1B6B1C6B1D6BD0
:102E30001E6B1F6B206B216B226B236B246B256B2E
:102E4000266B276B286B296B2A6B586B596B5E6B53
:102E50005F6B606B616B626B636B646B656B666B06
:102E6000676B686B696B6A6BD0500F0BD0A8000E54
:102E7000D080D082D088D886D8886B6FD180576BAD
:102E80000001B7EF03F0DEEF03F0F6EF03F087EF9A
:102E900004F0899897EF04F0899A899EF19CF29842
:102EA000F19AF096F198F098626A9AEF04F04F0E5A
:102EB000926EF70E936E370E616EF19E810E946ED8
:102EC000ACEF05F058C16CF159C16DF151EF06F04E
:102ED0005FC16DF15EC16CF157EF06F0050E0101A7
:102EE0009B6F00019EEC04F001C06CF101C06DF11C
:102EF0005DEF06F057EF07F0010E01019D6F000135
:102F00006EEC07F09D80EEEF07F085EF11F0030007
:020000040030CA
:0E00000000281E1E00B581000FC00FE00F404B
:00000001FF
